:100000000C943F020C9467020C9467020C946702F4
:100010000C9467020C9467020C9467020C946702BC
:100020000C9467020C9467020C9467020C94F71608
:100030000C9467020C9467020C9467020C9467029C
:100040000C94211B0C9467020C9467020C946702B9
:100050000C9467020C9467020C9467020C9467027C
:100060000C9472190C9467024E6F206D6173746565
:100070007200536C61766520646973636F6E6E65A0
:10008000637465640057726F6E6720736C61766588
:1000900020646174610031206D6173746572206D3C
:1000A000617800536C6176652070617573656400DA
:1000B000E700F50020736C6176652000206D6173A8
:1000C0007465722000506F6E67204D756C74697096
:1000D0006C6179657200506F6E67204D756C746944
:1000E000706C6179657200486F737420286D61735C
:1000F00074657229004A6F696E2028736C61766599
:10010000290003053F213F1208120A100A0E1C0E97
:100110000C1E0C141A14161F161E131E1E1B1E1E58
:100120001F1E3F213F3A2F3A173D173F213F181F0F
:1001300002040A041F0E04040E1F0A1F0A0E0E1FDB
:1001400004110E2E252E2F2A2E262929021F0208E1
:100150001F08150E04040E150E15151B151B04069D
:1001600004040C040000000017000300031F0A1F12
:1001700016371A1904130A153A000300000E11115C
:100180000E000A040A040E040030000404040010E7
:10019000001804031F111F121F101D151711151F22
:1001A00007041F17151D1F151D01011F1F151F1700
:1001B000151F000A00003200040A110A0A0A110A77
:1001C000040115020E11171E051E1F150A0E110A35
:1001D0001F110E1F15111F05010E111D1F041F11E8
:1001E0001F1108100F1F041B1F10101F061F1E04D5
:1001F0000F0E110E1F09060E112E1F051A121509DA
:10020000011F011F101F0F180F1F0C1F1B041B03C2
:100210001C03191513001F11030418111F000201FC
:10022000022020200001020C121E1F120C0C1212C0
:100230000C121F0C1A14041E05242A1E1F021C1463
:100240001D1020201D1F0814111F101E041E1E0249
:100250001C0C120C3E0A040C123E1E040214160A58
:10026000020F120E101E0E100E1E081E120C122669
:10027000281E322A26041E21001F00211E0401020E
:10028000013F213F0A4E6F20534420636172642076
:100290006F720A6E6F204C4F414445522E484558AC
:1002A0000A0A153A45786974001D20466C61736826
:1002B000696E670A20206C6F616465722E2E2E0AAB
:1002C0000A444F4E2754205455524E204F46462143
:1002D000000A0A153A49676E6F7265006D560A0A80
:1002E000504C45415345205455524E204F464620D0
:1002F000004C4F5720424154544552592120001779
:100300007361766500166261636B001574797065C0
:10031000000A0A0A153A6F6B617920163A6564691A
:100320007400596F7520656E74657265640A0054B7
:100330000A03E181867F3E186D830F0F0E018386CD
:100340006033186DC3198F1803C38E6033186DE3C3
:1003500030CF1803C39E603630CDE360CF3006C780
:100360009E7E3E30CDB360CF300CC6F6603330D9C0
:10037000B660CF33CFCCF66061B0DB1E60CF30D833
:100380006CE6C061B0DB1E618F19986CC6C063B1AA
:100390009B0E330F0FB078C6FF7E1F1B061E0F1774
:1003A000534400161378001613140015102000157E
:1003B00020100000000500893008023802497868E2
:1003C00014000045006801000005006801380100C4
:1003D000000500380168010000F6E8DBCFC3B8AEC5
:1003E000A49B928A827B746E68625C57524E494528
:1003F000413E3A3734312E2C29272523211F1D1C3D
:100400001A1917161514131211100F0E0D0C0B0AD2
:100410000908070618041C040101F7030101FF0382
:1004200000000000240027002A0000000000250032
:1004300028002B00000000002300260029000404EF
:10044000040404040404020202020202030303037C
:100450000303010204081020408001020408102058
:100460000102040810200000000700020100000340
:10047000040600000000000000006902E9171124D2
:100480001FBECFEFD8E0DEBFCDBF11E0A0E0B1E0EE
:10049000EAE6F3E402C005900D92AE32B107D9F757
:1004A00014E0AEE2B1E001C01D92A639B107E1F758
:1004B00014E0CEE7D4E004C02297FE010E94172189
:1004C000CA37D107C9F70E944F1D0C94B3210C9471
:1004D000000010927F0110927E018AE191E09093DA
:1004E0007D0180937C0180910D01992787FD909576
:1004F000E0E3F0E09F01281B390BC90162E070E0E6
:100500000E94C5206093B80184E590910F01891B7A
:100510008093BB0180911001992787FD90959F01E1
:10052000281B390BC90162E070E00E94C52060936E
:10053000BC0180910E018093BD01209111013327F0
:1005400027FD309584E590E0821B930B62E070E01C
:100550000E94C5206093BF01CF01821B930B62E014
:1005600070E00E94C5206093C00108958F929F9211
:10057000AF92BF92CF92DF92EF92FF920F931F93B1
:1005800080910B01882309F043C18091BF019091B4
:100590001201890F8093BF01909113018091C001D6
:1005A000890F8093C00187FF07C091959093130135
:1005B00083E591E00E94271720911101332727FD41
:1005C00030958091C001992787FD9095280F391F9C
:1005D000213331054CF080911301819580931301F3
:1005E00083E591E00E94271700911101112707FD73
:1005F00010956091BF01772767FD70954091C0010C
:10060000552747FD5095E090B901FF24E7FCF09491
:10061000C090B801DD24C7FCD094A0900C01BB248D
:10062000A7FCB09480900D01992487FC90948EE2F1
:1006300091E098010E94F40E882381F080910C01D2
:100640009091B901890F8093BF018091120181952A
:100650008093120183E591E00E9427170091110118
:10066000112707FD10956091BF01772767FD7095F1
:100670004091C001552747FD5095E090BB01FF24F4
:10068000E7FCF094C090BC01DD24C7FCD094A0909E
:100690000F01BB24A7FCB09480901001992487FC23
:1006A00090948EE291E098010E94F40E882381F0EC
:1006B0008091BB0190911101891B8093BF018091B2
:1006C000120181958093120183E591E00E94271722
:1006D0008091BF0187FF40C08091BE018F5F8093F2
:1006E000BE0183E591E00E9421172091110133277B
:1006F00027FD309584E590E0821B930B62E070E06B
:100700000E94C5206093BF0160E070E080E090E04F
:1007100022E030E040E050E00E94571F26E030E049
:1007200040E050E00E94922063506093120180915B
:100730001101992787FD909520E330E0281B390BA4
:10074000442737FD4095542F60E070E080E090E052
:100750000E94571F6093C00120911101332727FD8C
:1007600030958091BF01992787FD9095280F391FFB
:10077000253531050CF440C08091BA018F5F80931C
:10078000BA0183E591E00E942117209111013327DE
:1007900027FD309584E590E0821B930B62E070E0CA
:1007A0000E94C5206093BF0160E070E080E090E0AF
:1007B00022E030E040E050E00E94571F26E030E0A9
:1007C00040E050E00E9492206350609312018091BB
:1007D0001101992787FD909520E330E0281B390B04
:1007E000442737FD4095542F60E070E080E090E0B2
:1007F0000E94571F6093C0018091BA018A3020F493
:100800008091BE018A3020F01092BA011092BE0190
:100810001F910F91FF90EF90DF90CF90BF90AF901E
:100820009F908F900895EF92FF920F931F9382E015
:10083000809384018FE08093850110E110938601FD
:100840008CE7E82E81E0F82EC7016091BA014AE0FA
:1008500050E00E94871E89E38093850110938601F2
:10086000C7016091BE014AE050E00E94871E81E00E
:100870008093840100911101C7016091BF014091F3
:10088000C001202F0E946908C7016091B901409101
:10089000B80120910C0100910D010E946908C70167
:1008A0006091BB014091BC0120910F0100911001AA
:1008B0000E9469081F910F91FF90EF90089539C031
:1008C00083E194E00E9487178531F9F086312CF49A
:1008D0008A3041F0843169F50CC08E31E9F08F31F6
:1008E00041F521C083E194E00E9487178093BC0109
:1008F00020C083E194E00E948717909111019195A7
:100900009C5A981B9093BF0114C083E194E00E940D
:1009100087178093C0010DC083E194E00E94871780
:100920008093BE0106C083E194E00E948717809304
:10093000BA0183E194E00E947E17892B09F681E0D9
:100940008093B7011092B60108958AE08093C101A7
:100950008091B8018093C20180910B01882329F016
:1009600081E08093C1018093C2018091B501882309
:1009700029F082E08093C1018093C20121EC31E033
:10098000D9010D900020E9F71197A21BB30BE0915C
:100990001304F09114040280F381E02D83E194E0CC
:1009A000B901AD01099508951F9310920B0110E054
:1009B00016C061E070E080E090E00E949D1B1F5F28
:1009C000143169F48EE291E068E670E042E00E9442
:1009D000540E81E08093B60180930B0104C0809196
:1009E000B701882331F31092B7011F9108950F9337
:1009F0001F9303E114E0C80162E070E00E94A818B0
:100A0000C8016FE574E00E94DF17C80165EA74E071
:100A10000E94E4171F910F9108950F931F9303E114
:100A200014E0C80162E070E00E947417C8016AE037
:100A30000E9431186091B801772767FD7095C80151
:100A40000E943118C80164E10E9431186091BF0111
:100A5000772767FD7095C8010E943118C80165E1CC
:100A60000E9431186091C001772767FD7095C80119
:100A70000E943118C8016EE10E943118C8016091CE
:100A8000BA010E943118C8016FE10E943118C801F3
:100A90006091BE010E943118C8010E9474181F9114
:100AA0000F9108950F931F9383E194E062E070E04B
:100AB00042E050E00E9485188823C1F11092B601EF
:100AC00010920B0101E02BC083E194E00E94871794
:100AD000182F8230B1F08A3019F08130B9F407C094
:100AE00083E194E00E9487178093BC0118C08EE2D6
:100AF00091E063EA70E042E00E94540E10930B0113
:100B00000EC08EE291E066E970E004C08EE291E0F2
:100B100065E870E042E00E94540E00930B0183E10F
:100B200094E00E947E17892B79F60CC08EE291E04A
:100B300062E770E042E00E94540E81E080930B0176
:100B40008093B6011F910F9108950E9452050E9453
:100B5000B6020E940D05089583E194E00E94891871
:100B600008951F93CF93DF9311E010930B01109220
:100B7000B5011092BA011092BE018EE291E060EBD5
:100B800070E042E00E944711882319F0813079F427
:100B900007C010920B011092B6011093B5010DC061
:100BA00010920B011092B6011092B50106C08EE2B0
:100BB00091E065EC70E00E940C1411E0C0E3D0E01D
:100BC0008EE291E00E94D40F8823D1F388E391E074
:100BD00066E00E946407882309F05CC080910B01E5
:100BE0008823F1F588E391E061E041E00E946E071F
:100BF000882399F08091B801282F332727FD30955D
:100C000080910E01992787FD9095281B390B37FF9E
:100C100002C020E030E02093B80188E391E063E077
:100C200041E00E946E078823D9F080910D01992739
:100C300087FD9095AE01481B590B80910E01282F1E
:100C4000332727FD30958091B801992787FD90952E
:100C5000280F391F241735070CF4A9014093B80158
:100C6000109384018091B501882349F08CE791E0CD
:100C70006CEB70E00E94881D0E94A50508C08CE7FF
:100C800091E064EB70E00E94881D0E94D4040E94F1
:100C9000130496CFDF91CF911F9108950F931F9367
:100CA0000EE211E0C8010E941114C80166ED70E067
:100CB0000E940C14109246010E94AC050E94F70499
:100CC0001F910F910895882319F48CB5806202C09A
:100CD0008CB58F7D8CBD08959CB5937F982B9CBD62
:100CE00008952CB5382F33702C7F322B3CBD2DB599
:100CF00090E0959587959595879581702E7F822BAD
:100D00008DBD08958AE061E00E94EC1C8AE061E0FC
:100D10000E94801C8CB580618CBD8CB580648CBDBC
:100D20008DE061E00E94801C8BE061E00E94801CED
:100D30000895FC0181E08083089585E070E00E94C1
:100D4000201C08956F927F928F929F92AF92BF92D4
:100D5000CF92DF92EF92FF920F931F93CF93DF9387
:100D6000EC0189819A818C0124E0000F111F2A95E2
:100D7000E1F7081B190B85E10E94FE1BBC01600F07
:100D8000711F84E0769567958A95E1F77A83698388
:100D90008881882381F12E813F816217730710F4C7
:100DA000B90106C0888599858617970708F4BC01A4
:100DB00000D000D080E090E040E050E0E884F9848A
:100DC00000E010E0AD80BB24CC24DD246C807724CF
:100DD00088249924EDB7FEB761827282838294825F
:100DE0000E94EC1E6B830F900F900F900F9085E088
:100DF00070E00E94201CDF91CF911F910F91FF9016
:100E0000EF90DF90CF90BF90AF909F908F907F90AA
:100E10006F900895FC018CE39FE09383828384E0CC
:100E2000818381E084870895CF93DF93EC018C81E7
:100E30009D81892BB1F18C8590E08F719070892B09
:100E400069F584E10E94FE1BAA2797FDA095BA2FA1
:100E5000BC01CD010E94A31F26EE3FE34EEC50E4FF
:100E60000E942F200E94751F9B01AC017B836A8327
:100E70006115710589F084E08983B901FE0120E0E4
:100E8000848195816817790710F429830AC02F5F40
:100E900032962430A9F702C08FEF89838C858F5F4B
:100EA0008C87DF91CF910895FC0188E0808389E0F1
:100EB000818387E0828386E0838384E0848382E089
:100EC000858381E18683089520E0FC01E60FF11D12
:100ED0008781813009F421E0822F0895E62FF0E028
:100EE000423040F420E0E80FF91F878181508E3FA7
:100EF00088F40FC0E80FF91F87818F3F11F420E0BD
:100F000009C020E090E0642F70E00E94B1200197BA
:100F100009F421E0822F08950F931F93CF93DF935D
:100F2000EC0110E00FEF888162E00E94801C888154
:100F30000E941F1D2F81892B19F42F5F2F8307C05B
:100F4000222349F02F3F11F41F8201C00F838881B3
:100F500060E00E94801C1F5F2196173021F7DF910F
:100F6000CF911F910F910895FC01742F643508F003
:100F70006FC047FD6DC040330CF06AC080A1823065
:100F800021F5842F859585958595992787FD9095E1
:100F9000462F552747FD509524E530E0829FF0010C
:100FA000839FF00D929FF00D1124E40FF51FED5378
:100FB000FE4F808190E0272F277002C0959587957E
:100FC0002A95E2F78095817009C0833039F49485C1
:100FD000842F8627892780FF03C01FC08823E9F458
:100FE000E72FE595E595E59584E5E802F001112404
:100FF000862F992787FD9095E80FF91FED53FE4F37
:10100000777081E090E002C0880F991F7A95E2F72F
:1010100080952081282320830895E72FE595E59585
:10102000E59584E5E802F0011124862F992787FDD4
:101030009095E80FF91FED53FE4F777081E090E037
:1010400002C0880F991F7A95E2F72081282B208310
:101050000895FC0160A361A30895FC0160A341A36E
:101060000895EF92FF920F931F93CF93DF93EC01BC
:10107000E62EF42E022F10E007C0412F4F0DCE01B7
:101080006E2D0E94B4071F5F1017BCF3DF91CF9144
:101090001F910F91FF90EF900895EF92FF920F93A1
:1010A0001F93CF93DF93EC01E62EF42E022F10E076
:1010B00007C0612F6E0DCE014F2D0E94B4071F5F38
:1010C0001017BCF3DF91CF911F910F91FF90EF901C
:1010D00008959F92AF92BF92CF92DF92EF92FF92CC
:1010E0000F931F93CF93DF936C01962EB42EA22EF5
:1010F000C0E0D0E0E42EFF24E7FCF094112707FDC8
:1011000010950E0D1F1D06C0C601692D2A2D0E94C7
:101110004D0821964B2D4C0FCE018E0D9F1D801733
:10112000910794F3DF91CF911F910F91FF90EF9072
:10113000DF90CF90BF90AF909F9008952F923F92F5
:101140005F926F927F928F929F92AF92BF92CF9257
:10115000DF92EF92FF920F931F93DF93CF9300D014
:1011600000D000D0CDB7DEB79E838D83C62ED42E9F
:10117000EE24E394E21A8EEF289F502C1124842E43
:101180008A94962E9A94A42EA394B62EB394F22EFB
:10119000662423E0722E10E0C801847090709A8358
:1011A0008983F801E270F070FC83EB8398E0292ECC
:1011B000312C202231220170107054C0E7FC04C091
:1011C000FA94F2E05F0EE50C639489819A81892B91
:1011D00071F04F2D4D0D8D819E816B2D0E94B407B6
:1011E0006F2D6C0D8D819E814A2D0E94B407EB817D
:1011F000FC81EF2B71F04D2D4F198D819E816B2D50
:101200000E94B4076F2D6C0D8D819E81482D0E9428
:10121000B4072114310471F06C2D6F198D819E81FA
:101220004A2D0E94B4074F2D4D0D8D819E81692D51
:101230000E94B4070115110571F06C2D6F198D8195
:101240009E81482D0E94B4074D2D4F198D819E819E
:10125000692D0E94B407E70CF2E07F0E8A949A94FD
:10126000A394B3946F140CF4A9CF26960FB6F894F8
:10127000DEBF0FBECDBFCF91DF911F910F91FF90C9
:10128000EF90DF90CF90BF90AF909F908F907F9026
:101290006F905F903F902F9008954F925F926F9262
:1012A0007F928F929F92AF92BF92CF92DF92EF92F6
:1012B000FF920F931F93CF93DF93EC01A62E742E12
:1012C0009E2DFF24F394F21A8EEF289F802C112478
:1012D000B42EBA9453E0C52ECE0CE22EDD2443E0AA
:1012E000942E10E031E0432E512C40225122692EE1
:1012F00063940270107034C0F7FC04C0EA9482E07A
:10130000880EF80CD3944114510489F06D2D6A0DA8
:10131000472D4E192E2D220F260DCE010E94310889
:101320006E2D6A0DCE014B2D2C2D0E94310801151A
:10133000110589F06A2D6D19472D4E192E2D220F9A
:10134000260DCE010E9431086A2D6E19CE014B2D5B
:101350002C2D0E943108F90C82E0980EBA94C80E28
:10136000DE1454F2DF91CF911F910F91FF90EF9017
:10137000DF90CF90BF90AF909F908F907F906F90B5
:101380005F904F9008957F928F929F92AF92BF92FD
:10139000CF92DF92EF92FF920F931F936C01962EE4
:1013A000A42EF22E7E2C760E1EEFE19E102D11241F
:1013B000812E820E672D282D0E944D08B02EBA0C6A
:1013C000BA94C601672D4B2D282D0E944D08AE0CF6
:1013D000100FC601692D4A2D212F0E943108F90CEA
:1013E000FA94C6016F2D4A2D212F0E943108C601A3
:1013F000672D4A2D2E2D01E00E949E08FE18C60181
:101400006F2D4A2D2E2D02E00E949E08BE18C601A7
:101410006F2D4B2D2E2D04E00E949E08C601672DD6
:101420004B2D2E2D08E00E949E081F910F91FF90DA
:10143000EF90DF90CF90BF90AF909F908F907F9074
:1014400008958F929F92AF92BF92CF92DF92EF92C8
:10145000FF920F931F936C01162FA42E922EF02E45
:10146000BE2C8E2C860E2EEFE29EE02C11242E2D0B
:10147000290D682D0E946908AB0CFA94FE0C1150DE
:10148000190D1B19C601612F4A2D2B2D01E0EF2CE0
:101490000E944D09C601682D4A2D2B2D02E00E94A5
:1014A0004D091F910F91FF90EF90DF90CF90BF906B
:1014B000AF909F908F9008952F923F924F925F929E
:1014C0006F927F928F929F92AF92BF92CF92DF9254
:1014D000EF92FF920F931F93DF93CF9300D000D032
:1014E000CDB7DEB74C01D62E142FF9018491319679
:1014F00094913197D40190966C90B3E5B6170CF4A3
:1015000057C1482F552747FD5095A62EBB24A7FC51
:10151000B0942A014A0C5B1C141415040CF048C149
:1015200010330CF045C1092F212F332727FD3095AB
:10153000892F992787FD9095820F931F18161906FA
:101540000CF036C162E0E62EF12CEE0EFF1ECA0151
:10155000079668E070E00E94C520762E17FF0EC047
:10156000010F862F90E0FC01E29FC001E39F900DE8
:10157000F29F900D1124E81AF90A10E0802F9927A4
:1015800087FD9095212F332727FD3095820F931FDC
:10159000C19714F000E3011BD7FCDD24C20185359F
:1015A000910514F084E590E0C82ED4011C969C901F
:1015B0009126ED2DF0E0CF018A199B09AC0147700F
:1015C000507020E830E002C0359527954A95E2F743
:1015D000B22E68E070E00E94C520AB014E0D5F1D89
:1015E0005C834B83212F277081E090E0682F01C03E
:1015F000660F2A95EAF715951595159584E5180255
:10160000A00111244E0F5F1F4D535E4F8824202EE2
:10161000332427FC3094472C5524C4C0EB81FC8133
:101620002491F1E06F1629F5AB81BC817B2D022F4F
:101630007A011D2D1BC0872F90E0202F30E08223E0
:101640009323892B21F0F7018081862B8083872FBC
:1016500090E095958795782F882321F41196FD01C8
:10166000049170E81F5F0894E11CF11C1C1518F32D
:101670008DC0662059F5F62EF094AB81BC817B2D90
:10168000022F5A8349831D2D1EC0872F90E0202FE3
:1016900030E082239323892B29F0E981FA8180812C
:1016A0008F218083872F90E095958795782F8823C9
:1016B00021F41196FD01049170E81F5F89819A81E0
:1016C00001969A8389831C1500F360C093E0691624
:1016D00039F0AB81BC817B2D022F7A011D2D54C0C6
:1016E000A62EA094AB81BC817B2D022F5A83498307
:1016F0001D2DE92CFF2428C0872F90E0202F30E0FB
:1017000082239323892B79F0812F90E08E259F25CA
:10171000E981FA81908180FF02C0962B03C09A2153
:10172000E981FA819083872F90E095958795782FAE
:10173000882321F41196FD01049170E81F5F8981CF
:101740009A8101969A8389831C15B0F291E09926BB
:101750001DC0872F90E0202F30E082239323892B18
:1017600021F0F701808186278083872F90E095956F
:101770008795782F882321F41196FD01049170E854
:101780001F5F0894E11CF11C1C1518F3660F19F477
:101790004C5A5F4F61E083948B819C81840D951D31
:1017A0009C838B83882D90E0821593050CF436CFB3
:1017B0000F900F900F900F90CF91DF911F910F918D
:1017C000FF90EF90DF90CF90BF90AF909F908F9061
:1017D0007F906F905F904F903F902F900895DC0125
:1017E000FB0184918F5F14968C93149731968491AA
:1017F0008F5F15968C93159731965F96FC93EE93B9
:101800005E9708953F924F925F926F927F928F9270
:101810009F92AF92BF92CF92DF92EF92FF920F937F
:101820001F93CF93DF93EC01862EA42E422F102F0F
:1018300038A023E526170CF4ABC03FE23A150CF4B0
:10184000A7C0C02EDD248C8190E001979C01C29E30
:10185000C001C39E900DD29E900D1124262F3327D8
:1018600027FD3095820F931F181619060CF090C0B3
:101870008D8190E09C01C29EC001C39E900DD29EBE
:10188000900D11242A2D332727FD3095820F931FA9
:10189000181619060CF07CC09924442E55246DC0EE
:1018A0009C01215030404217530711F460E00EC0F4
:1018B000429EC001439E900D529E900D1124840FB4
:1018C000951FEE8DFF8DE80FF91F64914C9DC001AF
:1018D0004D9D900D5C9D900D1124682C680EBB24CD
:1018E000792C780C3FC0E62EFF2460FF19C0113020
:1018F00039F44B2D4A0DCE01672D0E94B4072EC03E
:101900002C9DC0012D9D900D3C9D900D11244A2DC4
:10191000480FCE01662D212F012F0E9469081EC09D
:1019200099A188A19817D1F098A3113039F44B2DC3
:101930004A0DCE01672D0E94B4070FC02C9DC00137
:101940002D9D900D3C9D900D11244A2D480FCE01E8
:10195000662D212F012F0E94690838A2F594E79483
:101960006E2DB3942B2D332727FD30958D8190E07C
:10197000281739070CF4B7CF9394492D552747FD05
:1019800050958C8190E0481759070CF489CF38A204
:10199000DF91CF911F910F91FF90EF90DF90CF904B
:1019A000BF90AF909F908F907F906F905F904F907F
:1019B0003F9008950F93CF93DF93EC01262F6A3069
:1019C00049F48D819885899F802D11249A85980FDF
:1019D0009A8726C06D3029F169854A8508850E945D
:1019E000020C9C816885969F402D11248985480FA3
:1019F00049878F818823A9F0552747FD5095699F16
:101A00009001112484E590E0821B930B84179507C5
:101A100044F49D81699F902D11248A85890F8A87BE
:101A2000198681E090E0DF91CF910F9108951F9387
:101A3000CF93DF93EC01162FF8948F8560E00E941E
:101A4000EC1C888918161CF460E00E94EC1C1EBD7A
:101A50000DB407FEFDCF8EB5888918161CF461E021
:101A60000E94EC1C7894DF91CF911F910895FF9212
:101A70000F931F93CF93DF93EC018C858F5F8C873F
:101A8000FF2400E010E06F2D6064CE010E94170D6E
:101A9000CE0160E80E94170D8F8561E00E94EC1C6A
:101AA000888918161CF460E00E94EC1CF801ED53C4
:101AB000FE4F90E080818EBD0DB407FEFDCF8EB548
:101AC0009F5F31969435B1F7888918161CF461E050
:101AD0000E94EC1CF3940C5A1F4F86E0F81699F6FE
:101AE000CE0160E40E94170DDF91CF911F910F91FD
:101AF000FF900895CF93DF93DC0188EF91E0E3EC52
:101B0000F1E0EF019C01199221503040E1F7199664
:101B10001C9219971A961C92DF91CF910895EF921B
:101B20000F93CF93DF93EC014E876D872F87E98A60
:101B3000088B81E0888788A319A28F83CE0162E099
:101B400071E00E94EF0B0E94820681E00E94630612
:101B500085E00E9471068CE00E946C068E8561E033
:101B60000E94801C8D8561E00E94801C8F8561E051
:101B70000E94801C898918161CF461E00E94801C58
:101B8000888918161CF461E00E94801C8989181647
:101B90006CF460E00E94EC1C6AE070E080E090E091
:101BA0000E949D1B898961E00E94EC1CED852E2F0F
:101BB000332727FD3095F901E25CFB4FE491F0E01B
:101BC000EE0FFF1FE65DFB4F859194919D8B8C8BF3
:101BD0002E5A3B4FF90184918B8FEE852E2F3327A0
:101BE00027FD3095F901E25CFB4FE491F0E0EE0F48
:101BF000FF1FE65DFB4F859194919B8B8A8B2E5A3C
:101C00003B4FF90184918A8FE8892E2F332727FDD6
:101C10003095F901E25CFB4FE491F0E0EE0FFF1F1D
:101C2000E65DFB4F859194919F8B8E8B2E5A3B4F97
:101C3000F90184918C8FEF852E2F332727FD309566
:101C4000F901E25CFB4FE491F0E0EE0FFF1FE65D6F
:101C5000FB4F85919491998F888F2E5A3B4FF901B4
:101C600084918D8FCE0161E20E94170DCE0164E157
:101C70000E94170D8B8587FF02C08FE78B876B85CE
:101C80006068CE010E94170DCE0160E20E94170D20
:101C9000CE016CE00E94170DCE010E94370DDF913E
:101CA000CF910F91EF900895FC01EC57FF4F619396
:101CB0007193445F40830895CF93DF93DC01E0E8A4
:101CC000F7E785919491ED01C75ADF4FAD01405977
:101CD0005F4F8150904C09F04EC0E6E9F7E7E49180
:101CE000E883E7E9F7E7E4911496EC931497E8E9C1
:101CF000F7E7E4911596EC931597E9E9F7E78591F5
:101D0000949117969C938E931697EBE9F7E785913C
:101D1000949119969C938E931897EDE9F7E7E491C7
:101D20009B96EC939B97EEE9F7E7E4919A96EC93F8
:101D30009A97EFE9F7E7E491EA01E883E0EAF7E749
:101D4000859194915D969C938E935C97E2EAF7E778
:101D5000859194915F969C938E935E97E4EAF7E762
:101D60008591949191969C938E939097E6EAF7E7EC
:101D70008591949132C08CE3888314961C921497B9
:101D80002FEF15962C93159780E293E017969C936E
:101D90008E93169784ED93E019969C938E931897E3
:101DA00081E09B968C939B979A968C939A97FA01D5
:101DB00020838CEA9DE05D969C938E935C978EEDDC
:101DC0009DE05F969C938E935E9784E79EE091964C
:101DD0009C938E9390978CE39FE093969C938E9325
:101DE0009297DF91CF9108958F929F92AF92BF9279
:101DF000CF92DF92EF92FF920F931F93DF93CF93D7
:101E0000CDB7DEB7260F371FE216F30694F4AE0CFB
:101E1000BF1C6A157B056CF4040F151FC016D10694
:101E200044F480E08C0C9D1C481559051CF481E09D
:101E300001C080E0CF91DF911F910F91FF90EF9053
:101E4000DF90CF90BF90AF909F908F900895EF92CA
:101E5000FF920F931F93CF93DF937C018C01025B62
:101E60001F4FC8010E947A0DC80169EA72E00E9402
:101E7000881DC8010E94370D83E00E94710680E032
:101E800091E0EEEFFFE3099584E590E0E80EF91E9E
:101E9000F7011082C80164E872E00E94D31DC801F6
:101EA0000E94370DE701CA54D040CE010E948C0732
:101EB000CE0164E00E946407882339F462E370E095
:101EC00080E090E00E949D1BF0CFDF91CF911F91A9
:101ED0000F91FF90EF900895AF92BF92CF92DF9253
:101EE000EF92FF920F931F93CF93DF93EC01CA57AA
:101EF000DF4F8881C658D040882309F44AC08C300F
:101F000010F010E002C01CE0181BCA5ADF4F81E03D
:101F10008883C655D0406EE4C62ED12CCC0EDD1E73
:101F2000C60160E00E94290853E5A52EB12CAC0E35
:101F3000BD1EF50100814DE2F42E4F2D401B410FD7
:101F40000D5FC60160E024E533E0E32E0E94210A24
:101F5000C60161E00E942908F5010081F01AF10E26
:101F60000D5FC60160E04F2D24E50E94C309C95AE8
:101F7000DF4F84E08993F5018081181B115D188380
:101F8000AC9669917991C6010E94881D8881815023
:101F90008883DF91CF911F910F91FF90EF90DF9099
:101FA000CF90BF90AF900895AF92BF92CF92DF9243
:101FB000EF92FF920F931F93CF93DF93EC01E0E832
:101FC000AE2EB12CA80EB91EF501E080F180028181
:101FD00013810E94691BE61AF70A080B190B7FE7A9
:101FE000C72ED12CCC0EDD1EF601808190E0A0E042
:101FF000B0E08E159F05A007B10708F081C08E01E3
:1020000005581F4FF80180819181A281B38100970B
:10201000A105B10509F474C00E94691BF601208175
:10202000620F711D811D911DF50160837183828393
:102030009383FE01EF58FF4F80819181A281B3818C
:102040000196A11DB11D80839183A283B383F80102
:1020500010821182128213820E94771BC958DF4FAF
:10206000688379838A839B83C757D040CE010E94BF
:10207000A206CE010A960E948C07CE0148960E94C5
:10208000140781E032C08E010B5D1F4FC8010E9412
:102090006415C8010E94DB15C8010E94BE16CE015E
:1020A0000E946C0FCE010E948D108E01025B1F4FAB
:1020B000C8010E94370DCC5ADF4F8881C455D040EB
:1020C000882319F4C8010E947A0D0E94771BC55815
:1020D000DF4F688379838A839B83249728813981A2
:1020E000621B730B7A936A9380E0DF91CF911F910B
:1020F0000F91FF90EF90DF90CF90BF90AF90089539
:10210000C558DF4F88819981AA81BB81CB57D040C8
:102110000097A105B10541F7B6CFBF92CF92DF92EC
:10212000EF92FF920F931F93CF93DF93EC018C8D6F
:102130009D8D892B09F4A1C08E01025B1F4FC80140
:1021400061E040E00E942D08FE01E95AFF4FCE5A9F
:10215000DF4F85E59881891B808326961882C855B4
:10216000D040698D613009F469C0613028F0888DF4
:10217000653008F07CC076C0CE0185960E941615A9
:10218000CA5ADF4F81E08883C655D040C80162E05B
:1021900071E00E94EF0B1D8E1C8ECC5ADF4F18820F
:1021A000C455D040AAE0CA2ED12CCC0EDD1EBC2EC8
:1021B000ED2EF8EAFF2ECE010E94D40F8823D9F32A
:1021C000C80161EF72E00E94881D6A8D7B8DC80195
:1021D0004AE050E00E94761EC8016CED72E00E9459
:1021E000881D6F2D62956F70C80170E04AE050E065
:1021F0000E94D91EC80161ED72E00E94881DC601CF
:1022000064E00E9464078823C1F5FA94A1F68B2D3F
:102210009E2D60E00E949D0683B7817F846083BF0E
:1022200083B7816083BF83B7816083BF889583B79D
:102230008E7F83BF83B78E7F83BFBDCFCF58DF4FE5
:1022400088819981AA81BB818F709070A070B070D5
:102250000897A105B10518F4C80167E00CC0C801D2
:1022600068E709C0882349F06B5FC80104C0882370
:1022700021F0C8016FE20E94AB1DDF91CF911F9149
:102280000F91FF90EF90DF90CF90BF9008952F9225
:102290003F924F925F926F927F928F929F92AF92F6
:1022A000BF92CF92DF92EF92FF920F931F93DF9333
:1022B000CF93CDB7DEB762970FB6F894DEBF0FBEEF
:1022C000CDBF6C016C837D834B8324E530E0C20E6F
:1022D000D31EF60110822CEA3FEFC20ED31E3AE065
:1022E000A32EB12CAC0CBD1C25E2222E312C2C0CC3
:1022F0003D1C9EE4492E512C4C0C5D1C10E080E3EB
:10230000782E66241A823FEF3983A601495A5F4F1F
:102310005F834E83C601885A9F4F99878887F6014D
:10232000EA5AFF4FFB87EA8796012B5A3F4F3D87BA
:102330002C8703E5802E912C8C0C9D1C5B81452FF6
:1023400050E05F874E878B818150888BC6010E9449
:10235000D40F8823D9F3C50164E00E946407882361
:1023600069F4C50165E00E946407882339F4C5015A
:1023700066E00E946407882309F4D3C0F401008159
:10238000C50164E00E946407882329F0C1010E940E
:102390001B171983CBC0C1010E942117C7C0C501FB
:1023A00063E044E00E946E07882321F01F5FC101B3
:1023B0000E942717C50161E044E00E946E07882350
:1023C00021F01150C1010E942717812F992787FD05
:1023D00090952E853F858217930711F410E002C077
:1023E00017FD1889F4018081819F902D11248C5F45
:1023F000682E691A28C0872D992787FD9095262D6C
:10240000332727FD3095821B930B0297D4F48981E3
:1024100062960FB6F894DEBF0FBECDBFCF91DF91AD
:102420001F910F91FF90EF90DF90CF90BF90AF90F2
:102430009F908F907F906F905F904F903F902F90E4
:102440000895F1E0FA83862D992787FD9095272D31
:10245000332727FD3095820F931F62E070E00E94C2
:10246000C520762EEE81FF811082E885F985608394
:1024700021E0EA85FB852083EC85FD8510822C8197
:102480003D81C9019A8B898B00E0E12EFF24E7FC96
:10249000F09420C0802F90E08E159F0569F423E012
:1024A000EE81FF812083F40180818E9D802D112497
:1024B000870DE885F9858083E989FA8965917491AA
:1024C000C2010E94D31D0F5F29893A892E5F3F4FB9
:1024D0003A8B298B3B810317E8F2C20160E00E942E
:1024E0002908F40140814E9D402D11244150470D93
:1024F000C20160E024E50E944D08C20161E00E9433
:102500002908F40100810E9D402D11244250470DF1
:102510000D5FC20160E024E5B3E0EB2E0E94C30929
:1025200015CFFA81FF2309F066CF39CF802F90E0D5
:10253000909581959F4F2E853F85AC01249FC001CA
:10254000259F900D349F900D1124AEEF6A2E680EDA
:1025500052CF2F923F924F925F926F927F928F92C3
:102560009F92AF92BF92CF92DF92EF92FF920F9322
:102570001F93DF93CF93CDB7DEB72B970FB6F894A9
:10258000DEBF0FBECDBF9B878A877A8369835C835A
:102590004B838C0100591F4FF8018081882309F477
:1025A00022C18A859B858A5A9F4F9B878A8781E0B3
:1025B000EA85FB85808312921292E455F040FB87F6
:1025C000EA87108E4EE4E42EF12CEE0EFF1EC701BA
:1025D00061E00E9429083AE0232E312C8A859B85F0
:1025E000280E391E25E2622E712C680E791EE981B3
:1025F000FA81F491FD83B7E58B2E912C880E991EFC
:10260000A8E5CA2ED12CC80ED91EF2E54F2E512CAA
:10261000480E591E8D5A9F4F9F838E83E1E7AE2E41
:10262000B12C8A859B85A80EB91E198708878A85D3
:102630009B850E94D40F8823D1F39D81992311F4A7
:1026400010E003C0EE81FF811081C70160E040E02F
:102650002FE233E00E945C0A8B819C81892B41F040
:10266000145FC70160E0412F2B813C810E945C0A0E
:10267000F40110828CE0F6018083C70169817A81C0
:102680000E94881DF201208130E0C901880F991F46
:10269000820F931F909581959F4F8D5AF4018083EF
:1026A000EE81FF81208130E0C901880F991F820FE0
:1026B000931F909581959F4F835DF6018083F5016F
:1026C000808184FF04C0C7016FEA73E003C0C701C3
:1026D0006BEA73E00E94D31DF201208130E0C90152
:1026E000880F991F820F931F909581959F4F8D5A48
:1026F000F4018083F60180818F5F8083EA85FB850A
:1027000082A5882321F0C70167EA73E003C0C701EF
:1027100063EA73E00E94D31DF201808190E09C0186
:10272000220F331F280F391F309521953F4F2D5A07
:10273000F4012083F60180818F5F8083C7016FE9F8
:1027400073E00E94D31DC10165E00E9464078823E5
:1027500051F0EA85FB8562A56F5FC3010E942D17CA
:10276000C3010E942717C10164E00E946407882307
:1027700099F4E885F9856081262F30E040E050E04B
:10278000F50180819181A281B38182179307A4070B
:10279000B50708F16F3FF9F08A859B8580599F4FF7
:1027A0009B878A878FEFEA85FB858083E057F0401F
:1027B000FB87EA87C30160E00E940B15C3010E94FA
:1027C0001B1781E0EA85FB85808F0DC08A859B857C
:1027D0000E94270F2CCFC10166E00E946407882366
:1027E00009F425CFF3CF2B960FB6F894DEBF0FBEBA
:1027F000CDBFCF91DF911F910F91FF90EF90DF90B0
:10280000CF90BF90AF909F908F907F906F905F9090
:102810004F903F902F90089540E050E00E94A91201
:102820000895AF92BF92CF92DF92EF920F93CF9322
:10283000DF936C018FE790E0C80ED91E82E3F601AA
:10284000808381E090E0A0E0B0E0B293A293929305
:1028500082936F0185EF9FEFC80ED91E8FEFF601AF
:10286000808380E99FEFC80ED91EC6010E945C0ECE
:10287000C6010E949906C6016FEF0E949D066AE09C
:10288000A62EB12CAC0CBD1CC5010E945407C5017D
:102890000E948C07C60148960E940A07C601825B07
:1028A0009F4F6DE04BE020E10FE05EE0E52E0E94DF
:1028B0008F0DE601A596CE010E943A17C50165E08D
:1028C0000E946407882329F0CE0160E00E942D1742
:1028D00006C0CE0165EB73E040E00E941A15DF915F
:1028E000CF910F91EF90DF90CF90BF90AF90089570
:1028F0000F93DC01002309F069C0623009F443C082
:10290000633030F4662359F0613009F05FC00DC0C8
:10291000633009F444C0643009F058C04CC04B30F7
:1029200008F04AE056964C9351C0842F90E0880FEF
:10293000991F1F962D913C915097280F391FF9012F
:102940008591949190969C938E935F97FC0145910D
:10295000549114968C911497849F602D1124919614
:102960006C939197252F3327862F90E028173907EE
:1029700008F4652F14968C911497689F802D11246C
:1029800092968C9323C014968C911497489F802D17
:10299000112459968C9359975A962C9317C01496D4
:1029A0008C911497489F802D11245B968C935B9794
:1029B0005C962C930BC014968C911497489F802D95
:1029C00011245D968C935D975E962C930F910895DC
:1029D000FC01222371F4648B8481489F802D112493
:1029E000858B15A214A213A281E0878B8093C40368
:1029F000108E0895FC01662369F4178A158A14A2C3
:102A000013A2108E1092C7031092C6031092C40333
:102A10001092B4000895CF93DF93EC01662319F46C
:102A20000E94FA141982DF91CF91089560E00E940C
:102A30000B1508950F931F93CF93DF93EC018B0138
:102A4000442371F460E00E940B151E870D871B8ADA
:102A50001A8A81E0898389E08E8B198E1B8E1D8EE8
:102A6000DF91CF911F910F910895CF93DF93EC01E8
:102A7000662339F58881882321F18981882309F526
:102A8000898590E0880F991FEF81F885E80FF91F7D
:102A9000859194912FEF8F3F920711F4188211C006
:102AA0009C8790E0880F991FEA85FB85E80FF91F46
:102AB00065917491CE0140E00E941A1589858F5F5F
:102AC0008987DF91CF91089560E00E9435150895C0
:102AD0000F93CF93DF93EC01662309F068C08981DF
:102AE000882309F464C08D89882309F060C0EA89CD
:102AF000FB89EE0FFF1F4D855E85E40FF51F2591C5
:102B000034912115310509F040C08989813031F4B3
:102B10001B8A1A8AFA012591349137C0198288815B
:102B2000882379F0CE0160E00E9435158A899B895F
:102B3000880F991FED85FE85E80FF91F25913491C7
:102B400024C0CE0160E00E94FA1431C0E6E0369560
:102B50002795EA95E1F76F70422F4F7175E0369532
:102B600027957A95E1F72051CE0100E00E94781474
:102B70008A899B8901969B8B8A8B880F991FED858B
:102B8000FE85E80FF91F25913491B9017695679577
:102B90007695679520FDDACF6F73432FCE0120E045
:102BA0000E94E8148A899B8901969B8B8A8BDF910E
:102BB000CF910F91089560E00E9468150895CF931A
:102BC000DF93EC01662309F0D6C08F89882309F4CE
:102BD000D2C08D89882321F4CE010E94FA14CBC083
:102BE00081508D8B8DA1882309F03BC08BA19CA1C6
:102BF0000196880F991FEF8DF8A1E80FF91F8591B5
:102C00009491282F27702EA3AC0163E05695479529
:102C10006A95E1F79A0136952795892F9927869528
:102C200086958FA32F738C81289F202D11242DA38F
:102C300041704093C8038BA19CA101969CA38BA3D8
:102C400029A130E08217930760F08AA1882329F038
:102C5000281B31093CA32BA304C0CE0160E00E94D5
:102C6000FA148DA181508DA3988D9F5F988F2FA10D
:102C70008C89280F8C85280F2A836B8D662369F039
:102C8000892F992787FD909570E00E94C5208C8D33
:102C9000869F802D1124820F8A838A8190E0CB96B3
:102CA0006BE370E00E94C5208A832E892B83698D97
:102CB000662379F0888D772767FD7095992787FDC2
:102CC00090950E94C5208A8D869F802D1124820FA9
:102CD0008B836D8D662399F0888D992787FD90955C
:102CE00070E00E94C520CB0162E070E00E94C52028
:102CF0009E8D899F802D11249B81890F8B838B81D1
:102D00008A300CF089E087FD80E08B838C898F33DB
:102D100009F41B82F894EA81F0E0E752FC4FE49159
:102D2000E093C5032D8130E08B81992787FD909535
:102D3000A901489F9001499F300D589F300D1124E3
:102D400088A590E0A901489F9001499F300D589FA8
:102D5000300D11248EA1992787FD9095AC01249FF9
:102D6000C001259F900D349F900D11248093C603C0
:102D70008093C7037894DF91CF91089560E00E941B
:102D8000DF1508956091C603662381F18091C30326
:102D90008F5F8093C3039091C503891738F130E0AA
:102DA0008091C403882309F431E03093C403109266
:102DB000C3038091C8038823A9F08091140123E400
:102DC000829FC0011124895B8093140190E070E020
:102DD0000E94B1208093C70305C08091C7038093F0
:102DE000B40008953323C9F780E0F9CF08951F9206
:102DF0000F920FB60F9211242F933F934F935F932F
:102E00006F937F938F939F93AF93BF93EF93FF93B2
:102E10000E94C216FF91EF91BF91AF919F918F9148
:102E20007F916F915F914F913F912F910F900FBEC6
:102E30000F901F90189561ED73E040E00E941A1505
:102E4000089569EC73E040E00E941A15089563EC60
:102E500073E040E00E941A150895FC01862F6681F8
:102E600070E06F5F7F4F992787FD90950E94C52086
:102E7000858308950F93FC0181E0848384E080A71B
:102E800084E194E0908B8787CF0161E040E020E00F
:102E900000E00E94781483E061E070E00E94201C52
:102EA000E1EBF0E08081887F81608083F89410926C
:102EB0008000E1E8F0E0108210928500109284001A
:102EC00088E191E0909389008093880080818860F8
:102ED0008083808181608083EFE6F0E08081826082
:102EE000808378940F91089581E080930E0460931D
:102EF000EB0310920C0410920D0408952091EA0344
:102F000030E08091E903281B3109C90108954091FF
:102F1000E9038091EA03481718F02FEF3FEF0AC04A
:102F2000E42FF0E0E753FC4F8081282F30E04F5F23
:102F30004093E903C9010895E091E9038091EA0310
:102F4000E81718F0EFEFFFEF06C0F0E0E753FC4F93
:102F50008081E82FF0E0CF0108950895AC01209121
:102F600011043091120421153105E1F09091E9032B
:102F70008091EA039817B0F090E008C0FA01EA0FD8
:102F8000FB1F8081A753BC4F8C939F5FA92FB0E09C
:102F9000A617B7079CF31092E9036093EA03CB01ED
:102FA000F90109950895E0910F04F091100430970C
:102FB00029F010920C0410920D0409950895709355
:102FC00012046093110408957093100460930F0429
:102FD0000895109216041092150488EE93E0A0E074
:102FE000B0E08093170490931804A0931904B09351
:102FF0001A0482E291E090931404809313040895DC
:10300000CF92DF92EF92FF920F931F93CF93DF93B4
:103010007C016B018A0180910E048823A1F0C0E03D
:10302000D0E00DC0D701ED91FC91D601AC0FBD1FD2
:103030000190F081E02DC7016C9109952196C01790
:10304000D10780F304C0CB01642F0E944D19C80141
:10305000DF91CF911F910F91FF90EF90DF90CF9074
:103060000895DF93CF930F92CDB7DEB7FC0169834C
:1030700080910E048823C9F080910D04803238F0CD
:1030800081E090E09383828320E030E015C080915E
:103090000C04E82FF0E0E451FC4F998190838F5F9E
:1030A00080930C0480930D0405C0CE01019661E06D
:1030B0000E944D1921E030E0C9010F90CF91DF91BE
:1030C00008950F93062F8091EB036CEE73E040910F
:1030D0000D0421E00E94F81810920C0410920D04C7
:1030E00010920E040F91089561E00E9461180895F6
:1030F000413208F040E2862F69EC73E00E94AF187D
:103100001092E9038093EA03089521E00E94781861
:1031100008951092E9031092EA0310920C041092A1
:103120000D040E94031B08950F931F938C01862F9B
:103130000E94AB1883ED97E10E946D198EEA97E12A
:103140000E946819C8010E9489181F910F91089563
:103150000E9494180895880F8093BA000895382F1C
:10316000413210F040E042C080911F048823E1F713
:1031700091E090931F04209321048FEF80938C049F
:10318000109247044150409348044F5F90932004AD
:1031900080912004330F832B80932004809122049C
:1031A000813041F410922204809120048093BB006E
:1031B00085EC01C085EE8093BC0080911F048130B6
:1031C000E1F380914704841710F44091470420E014
:1031D00030E00AC0FB01E20FF31FD901A95DBB4F2C
:1031E0008C9180832F5F3F4F2417A0F3842F089585
:1031F0000F931F93582F122F413210F081E04AC0D5
:1032000080911F048823E1F782E080931F040093DC
:1032100021048FEF80938C0410924704409348045C
:10322000A7E2B4E0FB0102C081918D938E2F861B33
:103230008417D0F31092200480912004550F852B21
:103240008093200480912204813041F41092220462
:10325000809120048093BB0085EC01C085EE8093B3
:10326000BC00112321F080911F048230E1F3809192
:103270008C048F3F11F480E00DC080918C0480326B
:1032800011F482E007C080918C04803311F084E057
:1032900001C083E01F910F910895482F613210F013
:1032A00081E0089580911F04843011F082E0089538
:1032B00060936A04A9E4B4E0842F9C01F90102C080
:1032C00081918D938E2F841B8617D0F380E0089513
:1032D000909326048093250408959093240480936A
:1032E000230408951F920F920FB60F9211242F936B
:1032F0003F934F935F936F937F938F939F93AF937E
:10330000BF93EF93FF938091B90090E0887F907016
:103310008036910509F4F2C081369105CCF58832EA
:10332000910509F47BC089329105B4F4803191058F
:1033300009F46FC0813191053CF4009709F447C14D
:10334000089709F04FC165C08831910509F466C03E
:10335000809709F047C182C08034910509F4A4C068
:103360008134910544F48033910509F482C0C897F3
:1033700009F038C189C08035910509F489C08835C4
:10338000910509F496C08834910509F02BC1AEC0AF
:103390008839910509F413C189399105ECF488370E
:1033A000910509F4ABC0893791054CF48836910535
:1033B00009F4A4C08037910509F014C19FC0883872
:1033C000910509F4FCC08039910509F49DC080384D
:1033D000910509F007C198C0803B910509F4C6C06A
:1033E000813B91054CF4803A910509F49FC0883ADD
:1033F000910509F0F7C0BAC0803C910509F4E3C01B
:10340000883C910509F4DFC0883B910509F0EAC0CA
:10341000C2C0809120048093BB00CFC0909147042C
:1034200080914804981768F490914704E92FF0E0E0
:10343000E95DFB4F80818093BB009F5F90934704C1
:10344000BCC080912104882309F44BC085ED809392
:10345000BC008091BC0084FDFCCFC2C080E28093A0
:103460008C0485ED8093BC008091BC0084FDFCCF72
:10347000B7C080E380938C0485ED8093BC0080917D
:10348000BC0084FDFCCFACC088E380938C049BC05F
:10349000809147049091BB00E82FF0E0E95DFB4F7D
:1034A00090838F5F809347049091470480914804F4
:1034B00082C0809147049091BB00E82FF0E0E95D65
:1034C000FB4F90838F5F8093470480912104882372
:1034D00041F085ED8093BC008091BC0084FDFCCF61
:1034E0007FC081E08093220484EA6EC085ED8093E2
:1034F000BC008091BC0084FDFCCF72C083E080934F
:103500001F0410928B0459C080918B04803208F004
:1035100056C080918B049091BB00E82FF0E0E559F4
:10352000FB4F90838F5F80938B0447C080918B0407
:10353000803230F4E0918B04F0E0E559FB4F1082CB
:1035400085ED8093BC008091BC0084FDFCCF10927F
:103550001F0460918B04E0912504F09126048BE612
:1035600094E070E0099510928B042DC084E0809364
:103570001F041092690410926A04E0912304F091F0
:103580002404099580916A04882329F481E08093BA
:103590006A041092490490916904E92FF0E0E75B16
:1035A000FB4F80818093BB009F5F90936904909153
:1035B000690480916A04981710F485EC01C085E8CD
:1035C0008093BC000FC085EC8093BC0009C01092B2
:1035D0008C0485ED8093BC008091BC0084FDFCCF01
:1035E00010921F04FF91EF91BF91AF919F918F9126
:1035F0007F916F915F914F913F912F910F900FBEEF
:103600000F901F90189510921F0481E08093210461
:103610001092220482E161E00E94EC1C83E161E0EF
:103620000E94EC1CE9EBF0E080818E7F808380813A
:103630008D7F808388E48093B80085E48093BC000C
:1036400008951F920F920FB60F9211242F933F935C
:103650008F939F93AF93BF93809191049091920425
:10366000A0919304B0919404309195040196A11D0A
:10367000B11D232F2D5F2D3720F02D570196A11D51
:10368000B11D209395048093910490939204A0938C
:103690009304B093940480918D0490918E04A09132
:1036A0008F04B09190040196A11DB11D80938D04EB
:1036B00090938E04A0938F04B0939004BF91AF9128
:1036C0009F918F913F912F910F900FBE0F901F9060
:1036D00018958FB7F89420919104309192044091FD
:1036E0009304509194048FBFB901CA0108959FB704
:1036F000F89420918D0430918E0440918F04509164
:10370000900486B5A89B06C08F3F21F02F5F3F4FE6
:103710004F4F5F4F9FBF542F432F322F2227280F29
:10372000311D411D511D82E0220F331F441F551FC3
:103730008A95D1F7B901CA010895EF92FF920F93CC
:103740001F93CF93DF937B018C010E94771BEB01CA
:103750000EC00E94771B6C1B7D0B685E7340C8F324
:103760000894E108F10801091109C851DC4FE1147E
:10377000F1040105110569F7DF91CF911F910F91B8
:10378000FF90EF900895789484B5826084BD84B5ED
:10379000816084BD85B5826085BD85B5816085BD4C
:1037A000EEE6F0E0808181608083E1E8F0E0108265
:1037B000808182608083808181608083E0E8F0E0A6
:1037C000808181608083E1EBF0E080818460808390
:1037D000E0EBF0E0808181608083EAE7F0E08081C7
:1037E0008460808380818260808380818160808327
:1037F0008081806880831092C1000895982F8E3058
:1038000008F09E509770809115018295880F880F5F
:10381000807C892B80937C0080917A0080648093E7
:103820007A0080917A0086FDFCCF2091780040914B
:103830007900942F80E030E0282B392BC9010895BE
:103840001F93CF93DF93182FEB0161E00E94801C40
:10385000209709F44AC0CF3FD10509F449C0E12FB0
:10386000F0E0EA59FB4F84918330C1F0843028F4B2
:10387000813051F08230B1F50CC0863019F18730BB
:1038800049F1843079F514C084B5806884BDC7BD22
:1038900033C084B5806284BDC8BD2EC080918000D5
:1038A000806880938000D0938900C093880024C0F2
:1038B00080918000806280938000D0938B00C093C1
:1038C0008A001AC08091B00080688093B000C093D5
:1038D000B30012C08091B00080628093B000C093AA
:1038E000B4000AC0C038D1051CF4812F60E002C0CA
:1038F000812F61E00E94EC1CDF91CF911F91089510
:10390000CF93DF93482F50E0CA018E5A9B4FFC01A2
:103910003491425C5B4FFA018491882369F190E015
:10392000880F991FFC01E05EFB4FA591B491FC014B
:10393000E65DFB4FC591D491662351F42FB7F894FF
:103940008C91932F909589238C93888189230BC028
:10395000623061F42FB7F8948C91932F909589235E
:103960008C938881832B88832FBF06C09FB7F894E0
:103970008C91832B8C939FBFDF91CF9108958330DF
:1039800071F0843028F48130A1F0823021F514C028
:103990008630B1F08730D1F08430E9F404C08091F2
:1039A00080008F7703C0809180008F7D809380009E
:1039B000089584B58F7702C084B58F7D84BD089546
:1039C0008091B0008F778093B00008958091B0000F
:1039D0008F7D8093B0000895FF920F931F93F62E72
:1039E000482F50E0CA018A599B4FFC012491CA011B
:1039F0008E5A9B4FFC011491425C5B4FFA0104917B
:103A00000023C9F0222319F0822F0E94BF1CE02F4F
:103A1000F0E0EE0FFF1FE65DFB4FA591B4919FB75D
:103A2000F894FF2021F48C911095812302C08C9191
:103A3000812B8C939FBF1F910F91FF9008950F933F
:103A40001F93482F50E0CA018A599B4FFC012491D3
:103A5000CA018E5A9B4FFC010491425C5B4FFA01F4
:103A60001491112319F420E030E015C0222319F03D
:103A7000822F0E94BF1C812F90E0880F991F8C5CC1
:103A80009B4FFC01A591B4918C9120E030E0802304
:103A900011F021E030E0C9011F910F910895CF93FB
:103AA000DF930E94C31B0E944E06C0E0D0E00E943C
:103AB000B1052097E1F30E940000F9CFCF92DF9289
:103AC000EF92FF920F931F93CF93DF937C016B01D3
:103AD0008A01C0E0D0E00FC0D6016D916D01D70121
:103AE000ED91FC910190F081E02DC7010995C80F7F
:103AF000D91F015010400115110571F7CE01DF915A
:103B0000CF911F910F91FF90EF90DF90CF9008958C
:103B1000EF92FF920F931F93CF93DF937C018B0162
:103B2000C0E0D0E0F8010F5F1F4F6491662359F0A9
:103B3000D701ED91FC910190F081E02DC70109952D
:103B4000C80FD91FEFCFCE01DF91CF911F910F91F9
:103B5000FF90EF900895DC01ED91FC910190F081D0
:103B6000E02D09950895EF92FF920F931F938C011A
:103B7000DC01ED91FC910190F081E02D6DE0099563
:103B80007C01D801ED91FC910190F081E02DC801FC
:103B90006AE009959C012E0D3F1DC9011F910F91EF
:103BA000FF90EF900895EF92FF920F931F937C0187
:103BB0000E94881D8C01C7010E94B31D9C01200F2B
:103BC000311FC9011F910F91FF90EF900895CF937E
:103BD000DF93EC016115710519F420E030E00FC0AE
:103BE000DB010D900020E9F71197A61BB70BE881C8
:103BF000F9810280F381E02DAD0109959C01C90195
:103C0000DF91CF9108954F925F927F928F929F9212
:103C1000AF92BF92CF92DF92EF92FF920F931F93DA
:103C2000DF93CF93CDB7DEB7A1970FB6F894DEBF81
:103C30000FBECDBF2C01742ECB01223008F42AE038
:103C400019A231E2C32ED12CCC0EDD1E822E992476
:103C5000AA24BB24672D752FA50194010E94D820AA
:103C600079018A01C801B701A50194010E9492203F
:103C7000472D461B0894C108D1084A3014F4405D12
:103C800001C0495CF6014083E114F104010511050E
:103C900021F07E2C5F2DC801DDCFC201B6010E944C
:103CA000E71DA1960FB6F894DEBF0FBECDBFCF9132
:103CB000DF911F910F91FF90EF90DF90CF90BF9019
:103CC000AF909F908F907F905F904F900895DC0110
:103CD0002115310541F4ED91FC910190F081E02D29
:103CE000642F099508950E94031E0895EF92FF9294
:103CF0000F931F939A017B0100E010E0B801A70128
:103D00000E94671E1F910F91FF90EF900895EF9210
:103D1000FF920F931F939A01E62EFF2400E010E01C
:103D2000B801A7010E94671E1F910F91FF90EF90AD
:103D30000895CF92DF92EF92FF920F931F93CF934C
:103D4000DF93EC016A017B012115310541F4E88123
:103D5000F9810190F081E02D642F09951FC02A3070
:103D60003105D1F477FF17C0E881F9810190F08126
:103D7000E02D6DE209958C0144275527BA014C19B5
:103D80005D096E097F09CE012AE00E94031E980199
:103D9000280F391F04C02AE00E94031E9C01C9019C
:103DA000DF91CF911F910F91FF90EF90DF90CF9017
:103DB0000895EF92FF920F931F937B019A010027C2
:103DC000F7FC0095102FB801A7010E94991E1F91C2
:103DD0000F91FF90EF9008952F923F924F925F9234
:103DE0006F927F928F929F92AF92BF92CF92DF920B
:103DF000EF92FF920F931F93DF93CF93CDB7DEB770
:103E00003B014C0119012A016D897E898F89988DAA
:103E10006A197B098C099D09621A730A840A950A3A
:103E2000A40193010E949220E218F30804091509E5
:103E3000A80197010E94FA202A0D3B1D4C1D5D1D13
:103E4000B901CA01CF91DF911F910F91FF90EF90BF
:103E5000DF90CF90BF90AF909F908F907F906F90AA
:103E60005F904F903F902F900895EF92FF920F93A5
:103E70001F937B018C01611571058105910529F462
